:0400000025C074C1E2
:1000040025C1FCCF72C1FACFF9CFF8CF9AC298C2FA
:10001400F5CFF4CFF3CFF2CFC2C2F0CF97C2EECF79
:10002400EDCF3F065B4F666D7D077F6F78730000F1
:10003400770145000A0062012600020071013000C8
:100044000500800132000000F894EE27ECBBF1E0DB
:10005400FBBFEBBFE5BFF8E1F1BDE1BD8DE0A2E080
:10006400BB27ED938A95E9F780E094E0A0E6ED9351
:100074000197E9F7E8E3F0E085919591009761F045
:10008400A591B59105901590BF01F00105900D92D1
:100094000197E1F7FB01F0CFEFE5EDBFE4E0EEBF40
:1000A400C0E6D1E000C0E0E0E8BBEFEFE7BBE0E092
:1000B400E5BBEEE3E4BBE0E0E2BBE0E2E1BBBAD2E5
:1000C400E0E0EFBDEEBDEDBDECBDE7BDE6BDEBBDD3
:1000D400EABDE9BDE8BDE2BDE5BDE4BDE3BDEBB706
:1000E400E06CEBBFEFE0E5BFE0ECEABFE5E4E9BFBD
:1000F400E0ECE7B9EEECE6B9EBE4E8B9E0E0E0BF48
:100104007894A0E0B0E08BD4E0938201F093830173
:10011400A0918201B0918301A53FE1E0BE0718F0F0
:10012400E2E8F1E08BD2A2E0B0E07DD4A4E8B1E053
:100134008AD2ED93FC93A0918401B0918501A536F8
:10014400E0E0BE0718F0E4E8F1E078D2E5E0E5BDD0
:10015400E0E0E4BDE0916001F0916101662777275A
:100164003ED3ADECBCEC8CE89FE3BED3DF01CB0106
:10017400EFE1F5EA6AED73E445D464D3AAE8B1E0AB
:10018400F5D2ED93FC93A0917A01A13019F45DD2DC
:1001940061D20BC0A0917C01A13039F4E0918A01B5
:1001A400F0918B0157D25BD25AD25DD26627772762
:1001B40016D3A4E1BEEA87E490E496D3A0E0B0E0CD
:1001C4008CE993E41FD43ED3A8E8B1E0CFD2ED93F9
:1001D400FC9349D2E536A0E0FA0731F4E4E8F1E013
:1001E400A4E6B0E0A083B1833ED2EF3FAFEFFA07BD
:1001F40019F4E4E8F1E022D228D2E43FA1E0FA07BE
:1002040031F4E2E8F1E0A4EFB1E0A083B1831DD2C0
:10021400EF3FAFEFFA0719F4E2E8F1E00FD2E09113
:100224008901F070AFEFB0E0F3D322D2E09378010C
:10023400E0918801F0918901E050F140A0E0B1E043
:10024400E7D316D2E093790185CFFFCFAA93BA936F
:10025400EA93FA93EFB7EA93A998E0917701E03033
:1002640051F5F3D108D2AE17BF07C8F4EED13597D4
:1002740002D206D210F4E1E001C0E0E0E0937A019A
:10028400E4D13A97F8D1AE17BF0738F0E5E0EEBDF8
:10029400EFEFEDBDE8EDECBD01C0A99A0BC0D5D1DF
:1002A4003596E9D1AE17BF0710F4E1E001C0E0E0F4
:1002B400E0937A0112C0D7D1E436A0E0FA0711F432
:1002C400A99A0BC0D0D1309741F0E4E0EEBDE091A3
:1002D4007801EDBDE0917901ECBDE991EFBFF991B1
:1002E400E991B991A991189518950A921A926A936D
:1002F4007A939A93AA93BA93EA93FA93EFB7EA9309
:10030400E5E0E5BDE6EEE4BDA0917E01AC3081F40C
:10031400E0E0E0937E01E0917F01E03011F49598F4
:1003240001C0959AE0917F013ED3E0937F0105C01F
:10033400E0917E01EF5FE0937E01A5D1AE0FE091E5
:100344007301B0E0A7FDBFEF7ED19AD109F451C08B
:10035400E0917501EF5FE0937501A0917501A43000
:1003640009F042C0E0E0E0937501E0917701E030EC
:1003740011F4E1E093D187D1EA0FE03061F4A09168
:100384007301A13019F48DD1319602C08AD131970D
:10039400FE93EE9329C0E13061F4A0917301A33080
:1003A40019F47FD1319602C07CD13197FE93EE933C
:1003B4001BC0E23061F4E0917301E03019F471D1B3
:1003C400319602C06ED13197FE93EE930DC0E330A7
:1003D40059F4A0917301A23019F463D1319602C08B
:1003E40060D13197FE93EE9368D14DD1EA0FE0933B
:1003F4007301E0917401EF5FE0937401A0917401C3
:10040400A53009F091C0E0E0E0937401A09160018F
:10041400B0916101AF3FE3E0BE0731F4E1E0E09366
:100424007701E2E03BD11BC0A0917701A13029F410
:10043400E0E0E093770132D140D1A0917601A13080
:1004440071F4A6E8B1E03FD1A0918601B091870193
:10045400AC3DE5E0BE0719F4E0E020D12ED139D15E
:10046400CDD2DF01E4E6F0E0A3D2E0936F0131D115
:100474006D917C91A0916F01E4E635D1E0937D010B
:10048400A0917D01B0E0EAE0F0E0A5D2E0936E0136
:1004940060917D017727A0916E01EAE024D1E09379
:1004A4006D01E0916F01E03019F4EAE0E0936F012F
:1004B400E0916E01E03039F4A0916F01AA3019F493
:1004C400EAE0E0936E0114D1BED0309749F4AA98C3
:1004D400AD9AE0917701B7D0EF58FE4F0CD122C00E
:1004E400E130A0E0FA0731F4AD98AC9AE0916D01E7
:1004F40007D118C0E230A0E0FA0731F4AC98AB9A07
:10050400E0916E01FDD00EC0E330A0E0FA0761F483
:10051400AB98AA9AE0916F0196D0EE59FE4FE08114
:10052400E8BBE0E0E0937001E991EFBFF991E99154
:10053400B991A99199917991699119900990189516
:100544001895EA93A99A76D0E99118958A939A9383
:10055400AA93BA93EA93FA93EFB7EA93A0E0B0E0D0
:100564005ED2DF0172D08CD021F06FD0A0E0B0E079
:1005740066D2A2E0B0E057D2AE2F75D0B0E080D002
:1005840029F0E0918401A2E0B0E061D2E991EFBFEB
:10059400F991E991B991A9919991899118950A9242
:1005A4001A929A93AA93BA93EA93FA93EFB7EA93B7
:1005B400E0ECE7B9A0918E01B0918F011A9719F57B
:1005C400E0E0E0938E01E0938F019ED0EAE0F0E05A
:1005D400EFD1E0936001F0936101E0E0E0938C01DE
:1005E400E0938D01E0917B01EF5FE0937B01A091AB
:1005F4007B01AF3F39F4E1E0E0937C01E0E0E0937C
:100604007B0101C02CD0E4B1F5B17ED0EA0FFB1F11
:10061400E0938C01F0938D01AEE8B1E054D0369AAA
:10062400E991EFBFF991E991B991A9919991199043
:1006340009901895E0E0E3BFE2BF0895A0E0B0E0C0
:10064400A083B1830895F0E00895E0918201F091D0
:1006540083010895E0938001F09381010895E0E01F
:10066400E0937C010895E0918401F091850108955F
:10067400EA1BFB0B0895A0918A01B0918B010895A8
:10068400EA17FB070895A0E08499A1E0E2E0EA9F5D
:10069400F001AE2FE0E08299E1E00895E093760165
:1006A4000895E0917601A0E8B1E0CDDFEE0FFF1FE1
:1006B400AE0FBF1FED91FD910895E0E0E093860138
:1006C400E09387010895ED91FD913196FE93EE93A9
:1006D4000895E0917601A0E8B1E0B5DFEE0FFF1FC9
:1006E400AE0FBF1F0895EA9FF001DF01FB01C0CFE9
:1006F400E09170010895E081E8BBFADFEF5F0895AF
:10070400A2DFEE59FE4FF7CFA0918C01B0918D017D
:100714000895552342F4503811F4E0FF04C0319693
:10072400691F791F6BF050E8572711F45F93CAC013
:100734005F3F31F0660F000C57956795752F08954C
:100744005F9300200AF0CAC0C3C050E8192E1522D6
:10075400880F991F9527550F879550E8072E052276
:10076400660F771F7527550F67950895689401C024
:10077400E8945F93F2DF703818F07F3F08F4A2C06A
:1007840056E1571BAAF4519558300EF4593030F005
:10079400EFEFFFEF6FEF7FE777F91AC07727552365
:1007A400B9F0EE0FFF1F661F771F5A95D1F710C0DF
:1007B4007727583028F0EF2FF62F672F5850F9CFAE
:1007C400552331F076956795F795E7955A95D1F7C6
:1007D40000200AF4DBD05F910895689401C0E89486
:1007E400309760407040B1F0002426F0772312F473
:1007F4000094CCD0172E7EE1112032F07A95EE0FC2
:10080400FF1F661F111CF9CFEF2FF62F612D5F9389
:100814008ADF5F9108954F93AF01FD01DA01AB01C7
:10082400BC01CA01402D012C142E4F910895EA0FEA
:10083400FB1F681F0895E095F0956095EF5FFF4FEB
:100844006F4F08955F9381DF903849F150E8152682
:10085400703821F1572F591B2BF112F4DCDFFACF3A
:10086400583118F0AA27BB278827583028F0AB2F17
:10087400B82F88275850F9CF552329F08695B79576
:10088400A7955A95D9F7502D512572F0D0DF38F439
:100894006795F795E795739513F420C0BCDF43DFA4
:1008A4005F910895D8F7FBCFEA1BFB0B680B51F05F
:1008B40010F40094C0DF662392F3EE0FFF1F661F4F
:1008C4007A95CBF7EE27FF27662777275F91089560
:1008D400EFEFFFEF6FE77FEF5F910895EFEFFFEF2B
:1008E4006FE77FE75F9108955F932FDF703851F3CF
:1008F400903841F301240894791F23F41CF3002059
:100904003AF3ECCF0F921F932F933F934F931127FA
:1009140022279927689FA0018F9F302D410D591FD1
:100924006B9F300D411D591F8E9F27D0BF9F25D02F
:100934006A9F23D0BE9F1DD0AF9F1BD0AE9F110DC9
:10094400291F391F491F591FE32FF42F652F522FD9
:100954004F913F912F911F910F9066232AF0550FCD
:10096400EE1FFF1F661F02C073954BF2D2DE5F912C
:100974000895100D211D391F02C0200D311D491F7E
:10098400591F0895F195E195F0400895F09560950B
:100994007095E195FF4F6F4F7F4F08956F2F660F4E
:1009A400660B762F0895EE23E1E009F0EE27089513
:1009B4000024112490E1AA0FBB1F001C111C0E1A65
:1009C4001F0A18F40E0E1F1E01C0A1609A9599F714
:1009D400FD01D001089504D0EBDF0EF4D3DF0895B8
:1009E400E894F7FF02C0CEDF6894B7FF06C0A09575
:1009F400B095119600F8039400FA0895ED91FC91D6
:100A040011970895182E862F612D192E972F712D69
:100A14001B2EBF2FF12D1A2EAE2FE12D0895119606
:100A240002D0FE2F1197E199FECFFF93FFB7F89400
:100A3400AEBBBFBBE09AEDB3FFBFFF91089507D0F3
:100A44001196EF93EF2F03D0EF9111970895E19B47
:100A540002C0A895FCCF9FB7F894AEBBBFBBE09A89
:100A64008DB3E81719F0EDBBE29AE19A9FBF0895A0
:00000001FF
